:020000040000FA
:06000000BEEF17F0120034
:0600080004EF08F01200F5
:060018000CEF08F01200DD
:06100000BEEF17F0120024
:061008004CEF16F012008F
:061018004EEF16F012007D
:06102A000300CC2F0000C2
:101030009900000005000000CA2F00009E0000007B
:1010400002000000C22F0000F802000008000000AB
:10105000F9EC0CF06A6A686A9F0E6B6EFB0E696EA3
:101060006D8C6D9C6E6AD4EC0CF0DF6ADF500B6EF9
:101070000C6A100E0B5C000E0C5810E2DF50040DD1
:10108000F3CFE9FFF4CFEAFF000EE926040EEA22CF
:10109000EE6AEE6AEE6AEE6ADF2AE8D7160E706E26
:1010A00068A604D0030E9EEC0CF0FAD70201DE6BAA
:1010B000E36BE46BE56B6D98080ED26F040ED36F93
:1010C000C46BC36BFCEF0CF0F9EC0CF00201C351E4
:1010D0000BE16D6A696A6DB602D06D86FCD70201BC
:1010E000010EC36F160E6F6EC30508E16DBA06D010
:1010F000686A696A69806988020EC36F6850040B68
:1011000004E06950040B01E065D86DB249D0685025
:10111000010B11E06950010B0EE09ADF0201040E91
:10112000C36F0401400E026F040E036F080E016FBF
:10113000006B8C0E00136850100B04E06950100B0C
:1011400001E042D86850400B08E06950400B05E0D0
:10115000BBEC16F0060E9EEC0CF06850200B04E081
:101160006950200B01E01ED86850020B06E0695060
:10117000020B03E0BCEC16F06A6A040E0201C35DC8
:101180000FE369A60DD0DF6A040EDF5C09E268A6F2
:1011900007D06CCFEBF2030ED1DB26D8DF2AF4D7D1
:1011A000FCEF0CF070A00DD0C5EC0CF0EF508008F7
:1011B00007E1CEDBEF50840803E1E7DB8C0EEF6E36
:1011C0007090050E9EEF0CF06984040EB7DB6D8203
:1011D000B9EF16F06D92BAEC16F0699468A403D0DA
:1011E000020EACDBFBD71200FD0E0201EB1519E17C
:1011F0007E0EEB15E8407F0B040DF3CFC6F2F4CF63
:10120000C7F2000EC627040EC723C6C2C8F2C7C263
:10121000C9F2C87565EC0DF002E117EF09F028EF8F
:1012200009F0FD0EEB15040801E11AD8120090DB5D
:10123000EF50800B02E08CDBEF6A0201DA6BDB6BB4
:10124000DF6BE06BDE6B96D8BDEC16F0E6EF0AF0D4
:10125000020E0201DB5D02E170EF0BF05CEF09F0C2
:10126000C8DB76DBEF50400B01E0010EDF6E0201C0
:10127000D275080EC35D09E142C46EFF6E500008CE
:1012800002E2100E01D0040EC36FDB0513E157EC30
:101290000DF0D4D9020E0201DA5D03E159DB840EB0
:1012A00007D0DF5003E154DBC80E02D051DB880EBB
:1012B000EF6E01D001D8A0D352EC0DF0030EE12661
:1012C000020E0201DB5D2CE16D50100B29E05DDBAD
:1012D000EE52EF500B6E0C6A080E0B1821E10C5009
:1012E0001FE165EC0DF01CE1BEDBEF50800B18E157
:1012F000BADBCCDBDF6ADF500B6E0C6A080E0B5CCE
:10130000000E0C5822E2DF507FDBDF50EA6A400F0C
:10131000E96E040EEA22E552E750EF6EDF2AEBD7C2
:10132000DB6BBADBEF6A040ED2190B6ED3C20CF082
:10133000010E0BC0DBFF020ED3C2DBFF010EDBCFC1
:10134000E9FF020EDBCFEAFFEF6A0201E3AF0CD048
:10135000E651E71107E005D0E7C2FAFF0201E651C6
:10136000F96EFADF0201E39F030EE15C02E2E16A3B
:10137000E552FCD204014051600BE842E842E842E9
:10138000E842E842000901E0120041510C0A43E042
:101390000B0A3FE00C0A31E0010A22E00B0A1EE0D2
:1013A000020A1CE0030A18E0080A10E0010A0CE037
:1013B0000F0A08E0030A01E012000201DE8F080EA6
:1013C000C36F120072EF0AF0C9EF0BF00201C40EF6
:1013D000DC6F020EDD6F0CD0ADEF0AF00CEF0AF0FF
:1013E00044510201DC6FDD6BC50EDC27020EDD23EC
:1013F000DE81010EDF6FDE8F12000201DE8F04013D
:101400004451EA6AC50FE96E020EEA2242C4EFFFB8
:101410001200BFEF16F0120045DB050EE1260401B5
:10142000420510E140511F0B00090CE10201DE8F63
:10143000030E0401415D04E10201010EEA6F02D0D6
:101440000201EA6B0401425147E140511F0B0208BF
:1014500043E144510F0B00093FE00201DE8F040E0F
:10146000DB6A020EF36E040EDBCFF4FFF350F45C84
:1014700033E2F4DA040EDBCFE6FF04014451800BC3
:1014800001E0010EC9DAE552E724A5DA030E415D59
:1014900003E163DA840E1CD044510F0B0C6A700F09
:1014A0000B6E0F0E0C22020E0BC0DBFF030E0CC0E6
:1014B000DBFF020EDBCFE9FF030EDBCFEAFFEE908E
:1014C000ED5244AF03D049DA400E02D046DAC80EDE
:1014D000EF6E040EDB2AC5D7050EE15C02E2E16A7D
:1014E000E55244D2800E0401405D36E10201C00E97
:1014F000DE6F04014351030A1EE0010A09E0030AFA
:1015000029E10201AE0EDC6F2D0EDD6F120E1FD031
:101510009ADA730EF6262E0E87DA020E0201F76AA9
:10152000DC25F66EDD51F7220900F5CFDFF20A0067
:10153000F5CFE0F2120087DA750EF6262E0E74DA79
:10154000DCC2F6FFDDC2F7FF0800F5500201DF6FD5
:10155000E06B12000201DE6B120004DA0401486B3A
:10156000496B40511F0B020A11E0030A0CE0010A0B
:101570001DE10201DE8F040148810201EA0516E146
:101580000401488313D00201DE8F10D00201DE8FE8
:1015900065DA04014451800B01E0010E3DDA1BDAEB
:1015A000DCD9EF50040B02E0010E486F0201DEAF00
:1015B00007D0480EDC6F040EDD6FDE81020EDF6F98
:1015C000020EE15C02E2E16AE552D0D16D980201BF
:1015D000DEBF07D0E3AF02D093DA28D05DDA840E05
:1015E00026D0E3BF2AD0040140AF23D00201DF514F
:1015F0000401465D0201E0510401475904E246C47A
:10160000DFF247C4E0F21AD80201010EDB6F8FD976
:10161000B6D9800EEF6EB9D9EE52080EEF6EB5D97D
:1016200035DAB3D9800EEF6E42DA92D9C80EEF6E7A
:101630001200020165DAC80EEF6E120093D90201A2
:10164000080EDF5D000EE0590DE2DFC2DEFFE0C2F2
:10165000DDFFDA5102E1010E03D0DA0506E1020EE8
:10166000DA6F03D0080EDE6EDD6A72D9EF9270D9A0
:10167000EF906ED9010EDB50EF126AD9EE52DFCF38
:10168000EFFF000EDB50DF5F010EDB50E05B480E2A
:10169000E86F040EE96FDEB10FD0DCD91BE0DCC2CD
:1016A000F6FFDDC2F7FFDC2B000EDD230800F5504E
:1016B00084D9F3E2DB06F1D7CDD90CE0DCC2E9FF37
:1016C000DDC2EAFFDC2B000EDD23EF5076D9F4E219
:1016D000DB06F2D7020EE15C02E2E16AE55246D196
:1016E00041D953D9EE52EFCFDFFFDFCF0BF00B50D4
:1016F0000201E45D000EE55903E2E4C2DFFF09D018
:10170000DF500B6E0C6AE850E45DE46F0C50E55955
:10171000E56F010EDB6ADF50F36E010EDBCFF4FFE5
:10172000F350F45C10E2010EDB506ED9E1C2E9FF28
:10173000E2C2EAFFE12B000EE223E552E750EF6E32
:10174000010EDB2AE8D7000ED880E455000EE555DF
:101750000CE2CAD91AD9EF50400B03E184D9C80E64
:1017600002D081D9880EEF6E0ED07DD98FD9E65187
:10177000E71107E005D0E7C2FAFF0201E651F96E72
:10178000FADF0201E39F020EE15C02E2E16AE55248
:10179000EDD00201DE8F08D9010EE66EE66AE66A38
:1017A000C50EE66E020E98D942C4C4F2040142513D
:1017B00004E10201100EC36F12000201200EC36F7C
:1017C000C0EF16F0CFD84AD9E5D8040DF3500B6E10
:1017D0000C6A020E0F0B05E0D8900C320B32E806B3
:1017E000FBE1D8900B360C36D8900B360C367FD9EF
:1017F0000B50EE260C50ED22B0D8EF9EFD0EDB50C4
:1018000002E159D901D05CD9EA22DECFEEFFDDCF6B
:10181000EDFFA3D8EF9CA1D8040EE926000EEA2222
:10182000EF8C020EE15C02E2E16AE5529FD09AD8A9
:10183000FE0EDB500C6A700F0B6E0F0EDFD8FD0E24
:10184000DB50E66E8AD8E552E750EE6EED6AFD0E8B
:10185000DBA402D0E66AF0D8FD0EDBA203D0010EB5
:10186000E66EEAD8020EE15C02E2E16AE5527ED061
:1018700079D8FE0EDB5004E10FD9840EEF6E05D04F
:1018800089D8F6D887D8010FF3D8020EE15C02E2BE
:10189000E16AE5526BD066D8FD0EDB5002E010D94C
:1018A00001D009D9EA22EECFDEFFEDCFDDFF55D81A
:1018B00032D9FB0EDBCFEEFFFC0EDBCFEDFF4DD8B8
:1018C000EE52FA0EDBCFEFFF400E47D8E850EF168E
:1018D000880E43D8E850EF12FD0EDB5002E0F0D83E
:1018E00001D0E9D8EA22EF74DECF0BF0DDCF0CF0A7
:1018F0000BC0F3FF0CC0F4FF020EE15C02E2E16AF0
:10190000E55234D0CFD8010EF36EFC0EDB5004E06C
:10191000D890F336E806FCE1F31C0B6EFD0EDBCF2E
:10192000E9FFFE0EDBCFEAFF0B50EF16E5D09BD8A8
:10193000EE52080EEF6E97D88BEF0DF0E66E680E44
:10194000E66E0F0EE66EDEDFE552E552E55212005E
:10195000D2C2E9FFD3C2EAFF1200DECFE9FFDDCF3A
:10196000EAFF12009FD8020EE1261200E16EC4D0F9
:10197000FE0EEA6ADB34FE0BEA36E96E1200400E18
:10198000EE6E040EED6E33EF0DF0C6C2E9FFC7C276
:10199000EAFF1200FD0EDB50E8240D6EFE0EDB5058
:1019A000040DF3500D241200020EE66EE66AE66A9C
:1019B000710EE66E0F0E6CEF0DF0E66EE8C2E9FFF9
:1019C000E9C2EAFFE82B000EE923E552E750EF6E8B
:1019D000DF06010E1200040DF4CF0CF088D8F3508E
:1019E000EE260C50ED221200480EEE6E040EED6E47
:1019F000120058D8E6521200E5527ED00C220BC0DD
:101A0000DEFF0CC0DDFF1200EA6A480FE96E040E2B
:101A1000EA22EF50E66E1200E8240D6E44510F0BDF
:101A2000040DF3500D241200F7220900F5CFDCF26B
:101A30000A00F5CFDDF21200FE0EDBCFE6FFC2DEBC
:101A4000E552E55212004251F66EF76AD890F6362A
:101A5000F73612004CD8EE50ED101200000EDE6E7C
:101A6000040EDD6E1200C8C2E9FFC9C2EAFF12000F
:101A7000040DF3CF0BF0F4CF0CF0000E0B26040E88
:101A8000BDDF840E6ADFE850EF12120044D8400E2A
:101A9000EE6E040EED6E12004ADF71DF8C0EEF6EFB
:101AA000A8EF0CF0D9CFE6FFE1CFD9FF120050DF4D
:101AB00032D8F4EF0CF05CDFCA0EE926020E1200F9
:101AC00057DFD20EE926020E12005FDFEF503C0B0B
:101AD000E842E8420D081200E66E8DEC17F00B6E3E
:101AE000050EE15E0B50120022DFF4EF0CF0D9CFAF
:101AF000E9FFDACFEAFF1200E552E7CFD9FF120083
:101B0000020EDB6F25DFEE52EF6A22DFC80EEF6EAA
:101B1000EBDF33EF0DF0020EE926000EEA22120091
:101B2000400EE66E000EE66E020EE66E52EC14F00B
:101B3000E552E552E55200090CE060C085F0020173
:101B4000F95103E085C0E6FF08D085C0E6FF5DDA05
:101B500005D00201F95104E0E66AABD9E552120062
:101B6000F95112E18B50800B0FE1FDC20BF0FEC268
:101B70000CF0FD07000EFE5B0B500C1005E1E66853
:101B8000CCEC17F0E55218D812008990898293683E
:101B900002DB898A00DB8CDAFEDA8998FCDA898636
:101BA000898491DA90DA8B9E8EDA8DDA8CDA8BDA90
:101BB0000201FD69FE6912008992899889968994CB
:101BC000899A936875DA8B8E120074DAE652FE0EEB
:101BD000DB50DF6EDF98DF9ADF9CDF9EFE0EDB902E
:101BE000DB92DB94DB96DB380F0BE76EFE0EE7CF64
:101BF000DBFFDB50B7DAF5CF7FF0DF50B3DAF5CF9C
:101C000080F0E5525CD2936889848986899840DAAD
:101C1000899889864DDA936A8A6A4ADA39DA200E17
:101C20008A6E46DA35DA44DA9368898841DA815077
:101C300012002EDA815012003DDA89848986899853
:101C400037DA936A8A6A24DAFE0EDB508A6E20DA6B
:101C50009368898834D22EDAE652DF6A8150DF6ECB
:101C600017DADF50E5522BD2560E0201005D10E16B
:101C7000560E015D0DE10001615111E10001740E8C
:101C8000626F2B0E636F0001030E41DA010E06D066
:101C90000001615104E119DA010E39DA616F0201C4
:101CA000F96B120007DA0201F95105E100C27AF07E
:101CB000010EF96F08D000C27BF0F96B7AC000F218
:101CC0007BC001F2D1DFFBD1F5D93EDA2CE1000176
:101CD00079512BDA01E62EDA17E3DF6ADF5025DAD5
:101CE00001E628DA02E26CDAF9D70201FA5104E0DF
:101CF0000001792B0201FA6B0001615101E1ECD97D
:101D00000001795110E10CD079517F080CE3DF6AB2
:101D1000010EDB50DF5C02E253DAFAD7EBD98B8E8F
:101D20000201100EF96F020EE15C02E2E16AE55277
:101D3000E16EC5D1BFD908DA2BE100017951F5D99F
:101D400001E6F8D917E3DF6ADF50EFD901E6F2D9EF
:101D500002E241DAF9D70201FA5104E00001792BDD
:101D60000201FA6B0001615101E1B6D9000179511C
:101D70000FE10BD079517F080BE3DF6A010EDB50D6
:101D8000DF5C02E228DAFAD7B5D90201100EF96F4A
:101D9000020EE15C02E2E16AE552E16E90D18AD97D
:101DA000030EE126020EDB6A520E02010125022516
:101DB0000325E76E020EE7CFDBFFDB50045D0AE090
:101DC0000001615104E181D9010EA1D9616F0201C5
:101DD000F96B24D002C2DFFF010E03C2DBFF01C298
:101DE00079F00001795104E179690201010EFA6F7D
:101DF000DF501F0806E30201FB6B030EF96F9ADF49
:101E00000DD0010EDBCFE6FFDFCFE6FF15DFE55299
:101E1000E5520201FB6B040EF96F56DF030EE15C25
:101E200002E2E16AE552E16E4AD1BDD9FE0EDB5015
:101E3000DF5C16E2010EDBCFF3FFDB2AF350EA6A28
:101E4000000FE96E020EEA22EF50E66E0201F85131
:101E5000F82BEA6A7A0FE96E000E71D9DF2AE6D70D
:101E6000020EE15C02E2E16AE552E16E28D19BD903
:101E7000FE0EDB50DF5C14E2010EDB50EA6A7A0FE3
:101E8000E96E000EEA22EF50E66E010EDB50EA6AC0
:101E9000000FE96E020E53D9010EDB2ADF2AE8D7C4
:101EA0000201F86B020EE15C02E2E16AE552E16ECA
:101EB00006D100D9E6520201F951100A01E18BD096
:101EC000190A01E176D0010A4FE00F0A32E0010A57
:101ED0002AE0020A23E0070A1BE0010A0CE0030AD9
:101EE00005E00001615101E08CD08AD0FE0EDBCF0D
:101EF000E6FFD8DE5CD0050EF85D02E32DD901D0F7
:101F000038D9050E0201F85D01E27DD025D97BD0DC
:101F10000001615101E077D00DDF75D00001615102
:101F200072E1D2DE70D0FE0EDBCFE6FF5CEC11F08A
:101F30003ED0FE0EDB5006E1EFD865E100016151B5
:101F400060E11AD0510E0201005D0AE10201080EA3
:101F5000F96F0001615157E1350EE66E2C0E26D067
:101F60000001615150E11FD0FE0EDB500BE1D4D8CF
:101F70004AE10001615145E1630EE66E2C0E06D97F
:101F8000E5523FD05A0E0201005D0AE10201090E3E
:101F9000F96F0001615137E17A0EE66E2B0E06D023
:101FA0000001615130E1630EE66E2C0EEFD8E55270
:101FB0002AD0A96AAA0EA86EA69EA69CA684550E33
:101FC000A76EAA0EA76EA682050EE66ECCEC17F0E1
:101FD000E552A69416D00001615115E1FCC240F211
:101FE0000001400E626F020E636F0001010E666F0A
:101FF0000001676F0001616F0201F96BFC6B03D098
:10200000D9D80201F96BE5525AD054D8E652DF6AAA
:1020100002010051410A2DE0310A38E0200A36E081
:10202000030A34E0240A32E02F0A30E00F0A19E0F4
:10203000250A2CE0200A0BE0040A04E000016151AB
:1020400025E123D0020E9BD821E30EDE1FD09DDDBB
:10205000040E95D802E3A3DE19D08BD80201020E3C
:1020600012D093DDFE0EDBCFE6FFF0EC10F0E55270
:102070000DD00001615105E1070EE66E2C0E86D8E9
:10208000E5520201070EF96F01D094D8E55217D03E
:1020900082D8899480D88984CBEF10F07ED8EA2248
:1020A000EF500201FC25FC6F00017907DF2A1200C6
:1020B0000A0E8CD0D9CFE6FFE1CFD9FF1200E5524E
:1020C000E7CFD9FF1200FE0E81D00001770E626FBC
:1020D0002B0E636F000112000001000E626F010EF3
:1020E000636F0001800E666F0001010E676F0001D3
:1020F000616F12000001000E626F010E636F010E2E
:10210000DBCF66F00001676F0001616F1200666F40
:102110000001676B00011200FF2B640EE66EA7EC56
:1021200017F0E5520201FF5112000B6E0C6AD890B5
:102130000C501200800E0B5C000E0C581200EA22AC
:10214000E552E750EF6E1200020EE126010E79C053
:10215000DBFF000161511200050EE66E88DEE552DC
:10216000CFEF0EF0F76A630FF66E2B0EF722080022
:102170001200FE0EDBCFE6FF58DEE5521200F36ED2
:10218000FE0EDBCFF4FFF350F45C1200E66EBDEC04
:1021900014F0E5521200010E19D0DF50EA6A000F68
:1021A000E96E010E120086DF020EE126010EDB6AE7
:1021B000DF6A12008ADF020EAADF010E616F1200D1
:1021C0004ADDE66EEADFBBDF4EEF10F0E66ECCECE8
:1021D00017F0E5521200E1DFEA22EF684EEF10F04F
:1021E00064DA030EE1260201FC6B0201FA6B040EB5
:1021F000F36EFE0EDBCFF4FFF350F45C56E3020106
:10220000060EF96F01C279F002C291F003C292F09A
:102210000001795104E179690201010EFA6F570E4C
:1022200002010125022503250201FC6F00019151E5
:1022300001E1ADD9200E0001915D0DE290510BE05E
:10224000C80EE66EA7EC17F0E552CAD9C0D8FF0851
:1022500002E10001906B200E0001915D01E177D950
:10226000040EDF6EFE0EDB50DF5C15E2DF5045DA58
:10227000010EEFCFDBFF200E0001915D06E3010EA2
:10228000DBCFE6FF7ED8E55202D0010EDB50E76ED1
:10229000020E27DAE7D70201FA5105E0020E00012B
:1022A0007925796F02D00001792B030EE15C02E2FF
:1022B000E16AE552E16EFED1F8D9060EE126030E81
:1022C000DB6AFE0EDB500001795D0CE1FE0EDB06E1
:1022D000DB5013DA020EEFCFDBFF010EF36E030EBD
:1022E000F3CFDBFFDF6AFE0EDB50DF5C15E2DF5071
:1022F00004DA040EEFCFDBFF200E0001915D06E350
:10230000040EDBCFE6FF3DD8E55202D0040EDB50D1
:10231000E76E050EE6D9E7D7030EDB5019E0020E93
:10232000DB500201FC5D14E1EED902E100019B6B80
:10233000000161511FE10001BC0E626F2F0E636F3F
:102340000001010E666F0001676B0001616F12D022
:10235000030EDB500FE0020EDB500201FC5D0AE0D1
:10236000FCC240F20001615101E1B3D9CCD902E1D4
:1023700000019B6B060EE15C02E2E16AE552E16E50
:1023800099D193D9FE0EDB50FF080AE100019B5161
:1023900007E08986DDD9CDD9D7D9FE0EDB5016D01E
:1023A00063D9A00E02DAFE0EDBCFE6FF92C0E6FF95
:1023B00091C0E6FF94D8E552E552E5520001010EC6
:1023C0009B6FFE0EDBCFE6FF64D8E55273D1D9CF09
:1023D000E6FFE1CFD9FFE6529368010EE66ECCEC42
:1023E00017F0E5528988010EE66ECCEC17F0E55245
:1023F0000000000000008150DF6E010EE66ECCECA4
:1024000017F0E5528998010EE66ECCEC17F0E55214
:10241000DF5000D0E552E552E7CFD9FF120045D991
:10242000FE0EDB50800BE76EFE0EE7CFDBFF90D990
:102430008150800B04E0FE0EDB50800806E08150E6
:10244000800B06E1FE0EDB5003E17ED9010E02D0C7
:102450007BD9000E2FD193687BD981AA02D074D981
:10246000010C72D9000C92D973D9A00E8114DF6EC1
:10247000FE0EDB50A00BE76EFE0EE7CFDBFFDB505E
:10248000DF5C03E161D9010E02D05ED9000EE55296
:1024900011D17CD9936800019A6BDF6A080EDF5C6A
:1024A00019E239D913E13ED911E1D5DF000910E075
:1024B00032D90EE137D90AE10001010E9A6F81CFBE
:1024C00040F2FE0EDBCF41F2F00E6AD980DF05D07C
:1024D000DF2AE4D70001020E9A6FE552EBD0E5D86F
:1024E00000019B5105E189988986898452D905D0DC
:1024F000898689881ED98998936A2ED99368DAD0FB
:10250000D4D889988996898414D90F0E3AD941D99B
:1025100023D989869368CED039D90F0EC16E926ABD
:1025200093689492898A89988986898441D999D8AF
:1025300000D9FE0EDB508A6E94D8FBD892D808D909
:1025400093688150DF6E00D9DF50E552B3D048D890
:102550003EDFFF0808E07FDF010808E1E66883DF6F
:10256000E552010813E10001906B1200E6687BDF81
:10257000E55200090BE12BDF0201406F00016151C0
:1025800001E1A7D8F00E0CD90201F96B120089986D
:102590006BD8800E0AD968D8300E02D90001010E1E
:1025A000906FFE0EC1EF13F0F1D85ED8900EDED81A
:1025B00064D801E183D8E5527DD0E8D8AA0ED6D8F8
:1025C000050EFCD8550EE66EAA0EE66E020EF6D883
:1025D000900ECCD8050E51D801E170D8E5526AD0E2
:1025E000898489968998010EE66ECCEC17F0E55245
:1025F0008994010EE66ECCEC17F0E5528984010E49
:10260000E66ECCEC17F0E55289988996936A010E34
:102610008A6E010EE66ECCEC17F0E5528994010E3D
:10262000E66ECCEC17F0E5528984010EE66ECCEC38
:1026300017F0E552200E8A6E0000010EE66ECCEC1B
:1026400017F0E5528994010EE66ECCEC17F0E552D6
:102650008984010EE66ECCEC17F0E5520000936819
:102660001200010EC1EF13F0AA0E9FD8550EE66EB0
:10267000AA0EE66E2A0EDEEF13F0A0D8E66A200E50
:10268000E66E4ADFE552E552DF6EDFCF40F2010E23
:10269000E66EE66A41DFE552E552DF6EDFCF41F2DA
:1026A000F00E7ED8000161511200D9CFE6FFE1CFD4
:1026B000D9FF1200E552E7CFD9FF12005BD8020E16
:1026C000666F0001010E676F0001616F0201F96B17
:1026D000120050D8010E666F0001676F0001616F34
:1026E0001200E7CFDBFF0001922BDB500201FC253B
:1026F000FC6F00017907DF2A1200EA6A000FE96E19
:10270000020EEA2212000201F96B0201FC6BFF0EBD
:102710000001915D1200FE0EDBCFE6FF80DEE55288
:1027200000091200FE0EDBCFE6FF9DDEE552000938
:10273000120097DF899495DF898431EF13F0E0DE92
:10274000E552E552E55212008CDF899831EF13F023
:1027500088DF898831EF13F084DF899A82DFFC0EED
:10276000DB508A6E7EDF898A31EF13F0E66E550EFC
:10277000E66E12000001400E626F020E636F0001F0
:102780001200E66ECCEC17F0E55212008EDFE65236
:1027900012000ED8CEDFFE0EDB508A6E99EF13F0DA
:1027A000E66EE66AE66A9FEF13F0E0DFDEEF13F015
:1027B000936AFD0EDB508A6E99EF13F0E66E9FEF81
:0227C00013F014
:0E27C200040140511F0B010801E012004051BC
:1027D000600BE842E842E842E842E842010801E0D2
:1027E0001200445103E0440501E012004151220A65
:1027F00031E0030A24E0010A15E0210A0DE0010A94
:1028000001E012000201710EDC6F000EDD6F080E98
:10281000DF6FE06BDE8121D00201710EDC6F000EF4
:10282000DD6F1BD046C4E4F247C4E5F20201D80EC6
:10283000E16F040EE26FE66BE76BE38F12000201BB
:10284000D80EDC6F040EDD6F070EDF6FE06BC10E7C
:10285000DE6F120042C46CF00201DE8F1200040130
:10286000D86BC20ED96F010EDA6FDB6BDC6BDD6BE0
:10287000080EDE6F0001616B606B1A0EE66E020ED1
:10288000E66E17EC0CF0E552E5521E0EE66E030EF6
:10289000E66E17EC0CF0E552E55246D900016A6B82
:1028A0006B6B12002CD90001606B6851691102E159
:1028B000000E05D034D9EF50800B01E0010E000965
:1028C0002DE1FC0EDBCF0BF02AD9EE52EF50D88071
:1028D0000B5405E224D9EE52FC0EEFCFDBFF606B08
:1028E000FC0EDB50605D19E26051EA6A580FE96E38
:1028F000040EEA22EF50E66E6051E76EFD0EDBCF6C
:10290000E9FFFE0EDBCFEAFFE750E926000EEA22E0
:10291000E552E750EF6E602BE3D706D90001605116
:10292000F3D0EDD80001615107E1E2D8FC0EDBCF16
:1029300066F0010E676F616FE7D00BD917E1BDD864
:10294000E7D802E10C500BE0010EDBCFE9FFDB2AF8
:10295000020EDBCFEAFF01E3DB2AEF50F1E1C8D83A
:10296000DFCF66F00001010E676F616F030EE15C5F
:1029700002E2E16AE552E16EC7D0EBD818E19DD8DA
:10298000C7D802E10C500CE0010EDBCFF6FFDB2ACA
:10299000020EDBCFF7FF01E3DB2A0800F550F0E180
:1029A000A7D8DFCF66F00001676B010E616F030EE1
:1029B000E15C02E2E16AE552E16EA6D0A0D8020E27
:1029C000E12600016A516B1102E1000E08D06AC0D5
:1029D000E9FF6BC0EAFFEF50800B01E0010E000938
:1029E0005CE1030E615D01E1616B615156E0020E35
:1029F000615D08E1E66A000EE66EE66AA2D80001B3
:102A0000030E43D0610542E1400E0B6E0C6A665125
:102A10000B5C000E0C5803E2400EDF6E02D066C065
:102A2000DFFFDF50665D666F980E646F040E656FA2
:102A3000010EDFCFDBFF67510BE1010EDB5012E02F
:102A400062C0F6FF63C0F7FF0800F55044D8F5D721
:102A5000010EDB5007E062C0E9FF63C0EAFFEF5000
:102A60003AD8F6D70001665111E16AC0E9FF6BC0A0
:102A7000EAFFEE52EF500B6E0C6A400E0B1804E1A9
:102A80000C5002E1020E01D0030E616FDFCFE6FFB2
:102A9000980EE66E040EE66E54D8020EE15C02E279
:102AA000E16AE552E16E30D0030EE66E4BEC0CF0BD
:102AB0000B6E050EE15E0B501200DF6AFD0EDBCFE0
:102AC00006F0FE0EDBCF07F0DE5206C0DEFF07C0C9
:102AD000DDFFDD52120064C0E9FF65C0EAFFEF6E62
:102AE000642B000E6523622B6323010EDB061200AC
:102AF000FD0EDBCF62F0FE0EDBCF63F01200D9CF0C
:102B0000E6FFE1CFD9FF1200E552E7CFD9FF12006F
:102B1000DF2ADF500B6E0C6AFF0E0B18120068C024
:102B2000E9FF69C0EAFF1200400EE66E580EE66E3D
:102B3000040EE66EE66AB8DFF3CF68F0F4CF69F012
:102B40001200010EE66EB0DFF3CF6AF0F4CF6BF047
:0E2B50001200D5DF030EE126000161511200D4
:022B5E001B5BFF
:102B6000324A003031323334353637383941424316
:102B700044454600011E323F3F000D0A2050757447
:102B800074696E672064657669636520696E746F29
:102B900020626F6F74206C6F61646572206D6F646A
:102BA000652E200D0A20446973636F6E6E65637431
:102BB0002066726F6D2048797065725465726D6918
:102BC0006E616C2066697273742E200D0A20526546
:102BD000706C75672064657669636520616E64203A
:102BE0007573652048494420626F6F746C6F61642F
:102BF000657220746F206C6F6164206669726D77F6
:102C0000617265200D0A001B5B324A200D0A2050BC
:102C100072657373205120746F20636F6E666972E2
:102C20006D20626F6F746C6F61646572206D6F648C
:102C300065200D0A001B5B324A200D0A2050726588
:102C40007373205A20746F20636F6E6669726D20F3
:102C5000626F6F746C6F61646572206D6F64652064
:102C60000D0A000D0A20426F6F746C6F616465720B
:102C7000206D6F64652063616E63656C6C65642EA6
:102C80002046726F6D2075736572206F72207469B3
:082C90006D6F7574200D0A0040
:082C980083D81100D8CFE4FF3E
:102CA000E0CFE4FFE46E7CD8E550E5CFE0FFE5CF70
:102CB000D8FF100008D864EC08F090EC0DF022D892
:102CC000DEEC14F0F8D70F0EC16E070EB46EF26A88
:102CD00028EC08F06CEF16F08B8E936A816A926A8A
:102CE000946A806A826A8B9E948494908B80949E6E
:102CF000929892969294929A899889968984898AD0
:102D00008B9E120004D8200E0201C35D1200000148
:102D10009E519F1104E1100E9E6F270E9F6F9E071C
:102D2000000E9F5B6DA204D09E519F1121E116D031
:102D30000201C3510AE0C30503E0020EC35D02E1D4
:102D40008B801200040EC35D02E18B901200100E06
:102D5000C35D06E100019E519F110AE18B701200D4
:102D6000200EC35D05E100019E519F1101E18B70B2
:102D700012001200120012001200E1EF13F0120014
:102D80002FEF14F06D840201080EC16F070EC26FA1
:102D9000C107000EC25BC151C211FAE16D9412006D
:0E2DA000DACFE4FFE652E552E5CFDAFF12008B
:022DAE00120110
:102DB000000202000008D8040A000100010200011C
:102DC00009024300020100C03209040000010202AE
:102DD000010005240010010424020205240600015C
:102DE000052401000107058203080002090401000F
:102DF000020A0000000705030240000007058302E5
:102E00004000000403090434034D006900630072AC
:102E1000006F0063006800690070002000540065C6
:102E200000630068006E006F006C006F006700793F
:102E300000200049006E0063002E00380343004468
:102E40000043002000520053002D003200330032B6
:102E500000200045004500430020004A00330020C8
:102E600000500072006F006700720061006D006525
:0B2E7000007200C02D032E072E3B2E29
:042E7C002A0EF66EB6
:102E8000100EF76E000EF86E00010900F5508B6F02
:102E90000900F5508C6F03E18B6701D03DD009002C
:102EA000F550866F0900F550876F0900F550886F5F
:102EB00009000900F550E96E0900F550EA6E0900B5
:102EC00009000900F550896F0900F5508A6F090063
:102ED0000900F6CF8DF0F7CF8EF0F8CF8FF086C0D7
:102EE000F6FF87C0F7FF88C0F8FF0001895302E1B1
:102EF0008A5307E00900F550EE6E8907F8E28A0769
:102F0000F9D78DC0F6FF8EC0F7FF8FC0F8FF000124
:0A2F10008B07000E8C5BBFD7120088
:062F1A00FE0EE3CFE9FF0B
:102F2000FF0EE3CFEAFFE9CFF3FFEACFF4FFFB0E9A
:102F3000E35003E1FC0EE35009E0FB0EE30602E27E
:0E2F4000FC0EE306FD0EE350EE6EF1D712001C
:022F4E00FF0E74
:102F5000E3500F6EEF0E01D0F30EE76EE72EAEEFEB
:102F600017F00C0E0E6EE76AE72EB4EF17F00E2E78
:0C2F7000B3EF17F00F2EACEF17F01200BB
:042F7C0013EE00F060
:102F800023EE00F0F86A0A9C3EEC17F0E0EC17F034
:082F90005AEC16F0FBD7120009
:082F9800FF0EE350E84E1200A9
:0E2FA000000000D000D000D0E82EFAD71200BA
:022FAE0000EE33
:0C2FB00000F00F0EEE6AEA62FDD712007E
:042FBC004F002100A1
:022FC0001200FD
:082FC200000000000000000007
:022FCA00000005
:042FCC000000000001
:012FD0000000
:020000040030CA
:0100000024DB
:010001000EF0
:0100020039C4
:010003001EDE
:010005008179
:010006008178
:010008000FE8
:01000900C036
:01000A000FE6
:01000B00E014
:01000C000FE4
:01000D0040B2
:00000001FF
